:0C0245000A103F065B4F666D7D077F6F5F
:02000B0021BB17
:1001BB00C0E0C0F0C083C082C0D075D008438CD8DB
:1001CB00438AF00528315FD0D0D082D083D0F0D0D5
:0201DB00E03210
:10009900D2AFD2A9438901D28C751FFFE4F5287527
:1000A9001E12F520F51D7521FFF522F5247529404D
:1000B900752A40752B40752C40C3E52864809481CE
:1000C900500411E080F3E4F52831255113515E31D4
:0700D900DD5152319680E277
:10015F000523E523C39464402DE4F523432205755D
:10016F001C32051DE51D943C401CE4F51D43220285
:10017F000520E520943C400EE4F520051EE51E9475
:07018F00184003E4F51E22F5
:1000E000751B087521FFE4F52DF52EE51BF4551F52
:1000F000F5B07429252EF8E6F5907F0A7E0031FBD5
:10010000E4F590E5B020E403852E21E51BC313F54B
:100110001B052EE52E7002052DC39404E52D648089
:04012000948040C7C0
:0101240022B8
:10012500E52230E634E52075F00A84741025F0F8F0
:10013500E6F529E52075F00A842410F8E6F52AE5A8
:100145001E75F00A84741025F0F8E6F52BE51E758A
:0A015500F00A842410F8E6F52C22CD
:10021300E52230E20D151CE51C6004432B802253BC
:0302230022FB2299
:1001DD00E521F46018E52220E713432280751A32D9
:0E01ED00E52124FD60050470044126513722EF
:0E023700432240051EE51EB41803E4F51E2206
:10022600432240E4F51D0520E520B43C03E4F52017
:0102360022A5
:0C025200E52230E706D51A0353227F2274
:10019600E52230E61F30E01C5322FEE51EB41307AD
:1001A600E5207003751F7FE51EB41508E520B41E13
:0501B60003751FFF228C
:09025E00E52CB43F03E4F52C2269
:1001FB00E4FDFCC3ED9FEE6480F8EC64809850073F
:07020B000DBD00010C80ECA9
:0102120022C9
:0300000002000DEE
:0C000D00787FE4F6D8FD75812E020054C7
:10001900020099E493A3F8E493A34003F68001F264
:1000290008DFF48029E493A3F85407240CC8C333E8
:10003900C4540F4420C8834004F456800146F6DFB7
:10004900E4800B0102040810204080900245E47E00
:10005900019360BCA3FF543F30E509541FFEE493AC
:10006900A360010ECF54C025E060A840B8E493A373
:10007900FAE493A3F8E493A3C8C582C8CAC583CA9E
:10008900F0A3C8C582C8CAC583CADFE9DEE780BE56
:0102510000AC
:00000001FF
